:03000000021048A3
:03000B000200A24E
:03002B000202CB03
:03005B0002041587
:030073000203EF96
:1000800002030406080C10182030406080040608A3
:100090000C10182030406080A0C005050D0502033B
:1000A0000302C2AFC0D0C0E020622C20680241B77A
:1000B0003066024177302F02E4730563C3740595FF
:1000C0002540F5956340F12069EE758A78E5257045
:1000D00003758A000202C485258AC262E525F47090
:1000E00002213E206802212B758B00D0E0D0D0C2C7
:1000F00097C295C293D2AF32C297C295C293740A87
:10010000D5E0FDE53C1420E21520E10D207D02D272
:1001100092307D02D29602013BD29402013B207DB7
:1001200002D296307D02D29202013B758B00D0E064
:10013000D0D0C297C295C293D2AF32758B00D0E0B7
:10014000D0D0D2AF3241B7E525600A207D02D297E8
:10015000307D02D293C29541B7E5256002D2952049
:100160007D02C293307D02C29741B7E525600A2027
:100170007D02D293307D02D297207D02C297307DDE
:1001800002C29341B7207D02C296307D02C2922006
:100190007D02C292307D02C296740AD5E0FDE5254B
:1001A000600A207D02D297307D02D293C29541B77A
:1001B000207D02C296307D02C292C294740AD5E0BC
:1001C000FDE525600A207D02D297307D02D293C2E0
:1001D0009541B7C294207D02C296307D02C29274CE
:1001E0000AD5E0FDE5256002D295207D02C293305C
:1001F0007D02C29741B7C294207D02C292307D0237
:10020000C296740AD5E0FDE5256002D295207D02F4
:10021000C293307D02C29741B7207D02C292307DE9
:1002200002C296C294740AD5E0FDE525600A207DDD
:1002300002D293307D02D297207D02C297307D0298
:10024000C29341B7207D02C292307D02C296207DCA
:1002500002C296307D02C292740AD5E0FDE52560A7
:100260000A207D02D293307D02D297207D02C29770
:10027000307D02C29341B730723DE53C20E21A2046
:10028000E129207D02C296307D02C292207D02C209
:1002900092307D02C2960202B720E1E6207D02C2C2
:1002A00096307D02C292C2940202B7C294207D02AF
:1002B000C292307D02C296E525F4F58A758B0075F1
:1002C0006300D262D0E0D0D0D2AF32C2AFC2AD5361
:1002D000E6EFC0D0C0E0D2D3D2AFC2CEE5296007EE
:1002E0002074461529612978007900E580307E0167
:1002F000F430E30278FF53DACF207E0343DA203074
:100300007E0343DA10C2D8C271E580307E01F4303A
:10031000E30279FFC3E89970CE3061037529182094
:1003200074037529188859D270E52A6004152A616A
:100330003920740543DA01C2D82070026194A859AB
:10034000206102C270207431C3E894F0400374F05D
:10035000F8E8C4540F28F87984B703026179C3130D
:10036000C3138721200802C313200A06C3C898F8C4
:10037000617928F8500374FFF8C3E895625003E5EB
:1003800062F8882230690AC3E522955E4003855EE3
:1003900022852224A824C3E524955E4002A85E8815
:1003A00025C3E52594404002D26420CF0CD0E0D094
:1003B000D0C2D343E610D2AD32C2CF7801E5296076
:1003C000053074021529C3E55994014005755C0098
:1003D00061E3755D00756400E55C2401F55C500324
:1003E000755CFFD0E0D0D0C2D343E610D2AD32C0AE
:1003F000D0C0E0C2AF53917F53E67FC260759100D9
:10040000C3E49550F594E49551F595759104D0E0C9
:10041000D0D0D2AF32C2AF53E6EFC2ADC0D0C0E051
:10042000C0F0D2D3D2AFA8FBA9FCC2D830710281F0
:100430007C53DACF207E0343DA10307E0343DA2088
:10044000D271E580307E01F420E302815388268951
:1004500027C1B853DACF207E0343DA20307E03432E
:10046000DA10C2D8C271307402C1A47800E58030BD
:0F0470007E01F430E302C1A48859C18B53DACF67
:10047F00207E0343DA20307E0343DA10C2712061FD
:10048F0002A14C53DACF207E0343DA10307E0343B0
:10049F00DA20C2D8D27188548955C3E89552F8E949
:1004AF009553F9E4FB7E027A00C3E8948CE994003B
:1004BF005005755800A13CC3E894C8E99400500852
:1004CF00E4D2E4FB7A0AA119C3E89468E9940150D5
:1004DF0008E4D2E3FB7A0FA119C3E894D0E99402A0
:1004EF005008E4D2E2FB7A1EA119C3E894A0E99464
:1004FF00055008E4D2E1FB7A3CA119C3E89498E9CE
:10050F0094085008E4D2E0FB7A787E00C3E8955651
:10051F00FCE99557FD30E708ECF42401FCEDF4FD00
:10052F00755800C3EC9AED9E500375580188568993
:10053F0057A854A955885289537802C18BC3E8959F
:10054F0026F8E99527F9307C02C16F307B02C16F25
:10055F00307A02C168207502A16FE9FDE8FCA18E17
:10056F00E9C313F9E813F8307902C168E9C313F945
:10057F00E813F8307802C168E9C313FDE813FC20D3
:10058F006126C3EC941CED94024002A1A5ED7018F6
:10059F00C3EC94C850120528C3E528940A5002C131
:1005AF00A4755900D270C1A4E52860021528740003
:1005BF00207F0B7888E67896B40302789EE624FABB
:1005CF00FEE43400FFC3EC9EFCED9FFD920878889B
:1005DF00E6B40327A2085009207D20C2AFD27DA127
:1005EF00F7307D17C2AFC27DC297C295C293C29634
:1005FF00C294C292206902D26BD2AFA2085017E602
:10060F00B4030DECF42401FCEDF43400FD020625D7
:10061F0078007900C16F7888E6B40315EC33FCEDF0
:10062F0033FDC3EC940AFCED9400FD50047C007D77
:10063F0000C3EC94FFED9400400678FF7900C16F82
:10064F00EC856FF0A4C5F0A2F733F87900400302F0
:10065F00068B78FF790002068BE9C313F9E813F8CC
:10066F00307C0EE9600278FFC3E81338F8E43400F9
:10067F00F9C3E894FFE99400400278FF8859D270DB
:10068F00206102C1A4741FF4552F4BF52FC274E4DF
:10069F002B7002D27475291830740375290A3061D2
:1006AF0002C1B820740353DAFE752A06307403753D
:1006BF002A0AD0F0D0E0D0D0C2D3D2AD43E6103268
:1006CF0079010206ED79030206ED790A0206ED794A
:1006DF001E0206ED79640206ED79C80206ED781761
:1006EF00E4D5E0FDD8FAD9F6227A147B7802071404
:1006FF007A107B8C0207147A0D7BB40207147A0BE5
:10070F007BC8020714AC257525017902B27DE4C2BE
:10071F0094D5E0FDE5256002D295D5E0FDC295D5D3
:10072F00E0FDD294D5E0FDE525600A207D02D29749
:10073F00307D02D293E570D5E0FD207D02C2973067
:10074F007D02C2937496D5E0FDD9C1EAF8D5E0FDDC
:10075F00D8FBDBB1C2948C2522C37C007D0075F0E1
:10076F000005F0EA33FAEB33FB50F6EB13FBEA1319
:10077F00FAC3E9FFE8FEE89AF8E99BF95004EFF9AC
:10078F00EEF8B3EC33FCED33FDD5F0DFEDF9ECF81B
:10079F0022E889F08A20D2D4F8A9F07B0030F70B39
:1007AF007BFFF42401F8E9F43400F9E88520F0A484
:1007BF00ADF0F8E98520F0A4AFF0FEED2EF974004E
:1007CF003FFA7C04C3EA13FAE913F9E813F8DCF4EF
:1007DF008BF030F70AE8F42401F8E9F43400F9E873
:1007EF0089F0C2D4F8A9F02222E547603BC3E53B6C
:1007FF0013F9E53A13F8C3E53E98F8E53F99F95038
:10080F000CC3E89480E994FF4016020833C3E894C0
:10081F007FE994005003020833787F790002083390
:10082F00788079FF8843894422E5476058E543255E
:10083F0040F8E5443541F9854420E4300701F435AB
:10084F0042FA30E709C3EA94F04015020875C3EA8B
:10085F00940F500302087578FF79FF7A0F0208751D
:0F086F00780079007AF0C3E524955E5006E52401
:10087E006009018EE54420E70D018EE54430E70660
:10088E00884089418A4222E54770030208F978A11F
:10089E00E6FAC3E54333F8E54433F91207A0E9302D
:1008AE00E70BC3E89480E994FF401301D0C3E894AA
:1008BE007FE99400500201D0787F790001D07880D2
:1008CE0079FFE820E715C3E52398F84009C3E894BB
:1008DE000140030208F778010208F7E8F424012525
:1008EE0023F840030208F778FF884522E547700396
:1008FE0002095C78A2E6FAA841A9421207A0E930E3
:10090E00E70CC3E89401E994FF4016020933C3E8EB
:10091E0094FFE99400500302093378FF790002092D
:10092E0033780179FFE920E715C3E54598F84009CA
:10093E00C3E89401400302095A780002095AE8F408
:10094E0024012545F8400302095A78FF88242278AD
:10095E00FFC264E52D5406702FD264C3E53B940AA2
:10096E004009C3E52594405002C264E53B6019740A
:10097E00FF853BF0848537F0A4F8C5F0600278FF60
:10098E00C3E895615002A861886022020A36788316
:10099E00E6F520120E6E75E8901206CF75E890E51A
:1009AE00E820ECFBA8BDA9BE120F04756B30756C68
:1009BE0000C3740013FD743013FC74302CFC7400EF
:1009CE003DFDECFAEDFBC3E89AE99B4014E56B2480
:1009DE0030F56BE56C3400F56CEA2CFAEB3DFB80E0
:1009EE00E5AE6BAF6CC3E56C13F9E56B13F8C3E9B9
:1009FE0013F9E813F8E56B28F569E56C39F56A7AB1
:100A0E0003C3E913F9E813F8DAF7AA201A70097587
:100A1E006B00756C00020A361AEA6008EE28FEEFCB
:100A2E0039FFDAF88E6B8F6C2275E890227883E6A8
:100A3E00FFE5E820ECF7A8BDA9BE056DC3E56D94F2
:100A4E00084052756D00E9FA79A0E76044EA700734
:100A5E00E56E601B020A71C3E8956E6010E56E507C
:100A6E0006600C14020A7D0460F9020A7DE56EF53B
:100A7E006EC394A8401B755EC0C394054013755E8B
:100A8E0080C39405400B755E40C394054003755EAC
:100A9E000075BB0122E55EF46002055EE56DB407EC
:100AAE000375BB1E22743279A387F0A4C5F0A2F79A
:100ABE0033F8C3E8955E4002A85E88228824882514
:100ACE00886122753A00753B7F2275C820A8CCA993
:100ADE00CD75C824AA38AB3988388939C3E89AF855
:100AEE00E99BF9AA3AAB3BAC3AAD3B7E047F02C31D
:100AFE00EB940440021E1FC3EB940840021E1FC35A
:100B0E00ED13FDEC13FCDEF7C3EA9CFAEB9DFBEF55
:100B1E006009C3E913F9E813F8DFF7EA28FAEB39AD
:100B2E00FB8A3A8B3B400122753AFF753BFF223020
:100B3E006002613D854C50854D51D26043E6802266
:100B4E007892E6FFC3E535948240010FC3E53594F4
:100B5E00A040010FC3EF940640027F057E021E30B7
:100B6E0072010EC3E53B940350060E0E3072010E59
:100B7E00C3E53B940250060E0E3072010EA93BA83F
:100B8E003A7A04C3E913F9E813F8DAF7C3E89EF8E2
:100B9E00E99400F94009C3E89402E99400500478FE
:100BAE0002E4F9E9FBE8FAC3E913FDE813FC884C0B
:100BBE00894DC3EF94036037EF20E00DE82CF8E980
:100BCE003DF9ECFAEDFB020BEAE828F8E939F9C336
:100BDE00E89402F8E99400F97A02E4FBC3EF940377
:100BEE00400D8A4E8B4F884889498C4A8D4B2288FE
:100BFE004E894F8A488B498C4A8D4B223060028138
:100C0E000AD26043E680E52D54066027A83AA93B38
:100C1E00E53494085006E820E002A94D759100C312
:100C2E00E498F594E499F595759104D26053917F0B
:100C3E0043E68022D265753D00752000020C55D228
:100C4E0065753D00752040E52D54066002C265D2E3
:100C5E00AF206005E53D60012278017A02C3E53BD5
:0F0C6E00940540027802C3E53B940A40027803E4
:100C7D00C3E53B940F40027A03306904781E7A0174
:100C8D00206007E53D6003D2AF22D2AF0000C2AFB6
:100C9D00C3E53BFB940F40027B0FEB043073012344
:100CAD0020620123F93069027982E58BC39940D026
:100CBD00053DEAFBE59E7005E59B020CCCE59A54DB
:100CCD0040B52004DBEE81F92065028155C26575C2
:100CDD009100AE3AAF3BC3E49EF594E49FF5957554
:100CED009104D26053917F43E68081553065028136
:100CFD0055D88DD2AF2230690B053420601675346E
:100D0D0000020D2120600D20650A206B071581154D
:100D1D008102153022A84EA94F75910053917FC3C2
:100D2D00E498F594E499F5957591048548508549B5
:100D3D0051D26043E6802278003064053065027838
:100D4D0001E53575F007A4F9E5F028F5F0E9A2F015
:100D5D0013A2F113A2F213F535C394785003753530
:100D6D0078C3E53595364008D266C297C295C293D1
:100D7D00306002A17D854A50854B51D26043E6809B
:100D8D0022C2AFC296C294C29230720B90021974F5
:100D9D000AD5E0FD020DA4207D02D296307D02D24F
:100DAD0092759F33759E00753C02020EE9C2AF200D
:100DBD007D02C293307D02C2973072179001F6C248
:100DCD0094207D02C292307D02C296740AD5E0FD58
:100DDD00020DE3900159306206E5256002D295209F
:100DED007D03759E22307D03759E23753C03020E97
:100DFD00E9C2AFC296C294C29230720B9001D37405
:100E0D000AD5E0FD020E14207D02D292307D02D271
:100E1D0096207D03759E23307D03759E22753C04BF
:100E2D00020EE9C2AFC2953072179001B0207D025B
:100E3D00C296307D02C292C294740AD5E0FD020EB4
:100E4D005190014730620EE525600A207D02D29750
:100E5D00307D02D293759F33759E00753C05020E51
:100E6D00E9C2AFC296C294C29230720B90018574E2
:100E7D000AD5E0FD020E84D294207D03759E2230AA
:100E8D007D03759E23753C06020EE9C2AF207D02DF
:100E9D00C297307D02C29330721F900244207D02B2
:100EAD00C296307D02C292207D02C292307D02C276
:100EBD0096740AD5E0FD020EC990016B30620EE505
:100ECD0025600A207D02D293307D02D297207D03CA
:100EDD00759E23307D03759E22753C01306B131278
:100EED000F04740AD5E0FD740AD5E0FDD296D294B4
:100EFD00D292C266D2AF22900145C297C295C293DB
:100F0D00C296C294C292C26222788076FF0876FFA2
:100F1D000876FF0876FF0876030876040876080839
:100F2D007601087601087601788C76010876FF083F
:100F3D0076FF0876FF0876FF0876FF0876030876B9
:100F4D00FF0876FF0876FF0876250876D00876FA32
:100F5D000876FA0876040876FF0876010876000808
:100F6D00767A0876FF087601227887E6FFC27278D6
:100F7D0088E6C394036008C27DE630E102D27DC2EB
:100F8D007E7889E630E102D27EC3EF940260087567
:100F9D008E01D273020FA9758E00C273227880E67E
:100FAD00149000809378A1F67881E61490008093D8
:100FBD0078A2F6F104227886E61490008D9378A33A
:100FCD00F6F1042222789CE67536FF75370CB402D3
:100FDD00067536A075370AB4030675368275370562
:100FED0022227896E6FA7897E6FB307F047A007B2A
:100FFD00FFC3EB9AFCC3948250027C82756F00058F
:10100D006FEC856FF0A4C3E5F0948040F222D27F9F
:10101D00120FEF1206DE7A007B007C101206D4E56B
:10102D00592AFA74003BFBDCF37C04C3EB13FBEA97
:10103D0013FADCF7FEC27F120FEF22E5EF20E60375
:10104D007520000520903DFFE520146006901FFFE0
:10105D001460009304600375EF12C2D353D9BF75AA
:0E106D0081C043FF801206CF75EF0243B2032D
:10107B00E5B3240420E702F5B3120F04758008755D
:10108B00A40075F1FF75D4F775900275A5FC75F288
:10109B00FD75D50075A0FF75A60075F30075D6001C
:1010AB0075B0FF75A70175F4FF75E241120F1612AB
:1010BB00156278988670C2AF1206E81206F812060F
:1010CB00DE1206FF1206DE1207061206DE12167677
:1010DB001206E81206E81206E3C2AFE4F8F6D8FDF2
:1010EB0078C879C8308307D9FBD8F7021C00120FD8
:1010FB0016121562120F76120FAA120FC3120FD10E
:10110B00120FD2120FEE120FEF78988670120F0497
:10111B0075885075891275C82475910475D84075FA
:10112B00A82275B80275E690759B80759D00759A1F
:10113B0080759C0075D10E75BC5875BB0175BA1FB7
:10114B0075E8801206CFD2AF12099943DA01C2D8E3
:10115B00C2711206E8753001D2617B037A0CE55837
:10116B0070067A0CDB0201E41206DE20700201E449
:10117B00C270E559C3940240E3E52F541F855B5AB7
:10118B00F55BB55AD7DAD7C26153DACF207E03436A
:10119B00DA20307E0343DA10C2D8C271C2757528CB
:1011AB00001206E3307409C3E528940A4002D27595
:1011BB001206D478023074027800C3E5599840F0D7
:1011CB00C2AF1206F81206F81206F8D2AF1206E8F2
:1011DB007546007888E6B4030241BF1206D4788CBA
:1011EB00E6C3940150030212BFE530C394015003D0
:1011FB000212BF207435C3E55994FF50030212BF8E
:10120B00C2AF12070DD2AF1206E3C3E559940150DA
:10121B00EFC2AF1206F81206D91206F8D2AF1206B9
:10122B00E3C3E55994FF40E90216FB7F05D27F1219
:10123B000FEF1206E3C2AFC27F120FEFAE59C3E539
:10124B0059947FD2AF40771206CFC2AF12070DD29F
:10125B00AFDFDA111BC3EE94057897F61206E8128E
:10126B0015A412167E7F0AD27F120FEF1206E3C26D
:10127B00AFC27F120FEFAE59C3E559947FD2AF5077
:10128B00E41206CFC2AF1206F81206D91206F8D234
:10129B00AFDFD4111BEE24057896F61206E8121573
:1012AB00A41216AD1206E3120FEFC3E55994FF40DB
:1012BB00F30216FBC3E559954640038559461206C2
:1012CB00E378017988E7B403027805C3E5599840C0
:1012DB000221DEC2AF12070D12070D12070DD2AF9E
:1012EB001206E8753000E4F531F5320531E531F4DD
:1012FB0070390532789AE6781914601278321460D6
:10130B000D787D14600878FA146003753200C3E51C
:10131B003298401715327531B478998670C2AF1276
:10132B00070DD2AF789886701206E31206D9E5291D
:10133B00700530740201E478012074027806C3E56D
:10134B00599840A77888E6C3940360031206E3E537
:10135B0029700201E4C2AF120F04E4F522F523F564
:10136B0024F525D2AF78858662F53EF53FF540F53D
:10137B0041F542F56DF547F52CF52DF535120AD1F2
:10138B00756D0875BB1E1206CF120A37E5E820EC07
:10139B00FBA8BDA9BEE97001F8886E120A3B756DFA
:1013AB000875BB1E7887E6FE7602120F767887EEFD
:1013BB00F6C2AF755EFF120AB385225E85225F858A
:1013CB002260D2AF752201752401752501855D64FC
:1013DB00756501D268D269753400120E6E120E98C3
:1013EB00120AD1120AD8120B4E021403120F041256
:1013FB000F76756D0075BB01120C4D120D03120D9E
:10140B00221207F7120D44120D8E120AD8120B3D41
:10141B00120B4E120C0A120C42120D03120D221259
:10142B0007F812095D120D44120DBA120AD8120BED
:10143B003D120B4E120C0A120C4D120D03120D2203
:10144B00120838120D44120DFE120AD8120B3D125F
:10145B000B4E120C0A120C42120D03120D22120823
:0D146B0095120D44120E30120AD8120B3DDE
:10147800120B4E120C0A120C4D120D03120D2212F1
:1014880008FA120D44120E6E120AD8120B3D120BF6
:101498004E120C0A120C42120A37120D03120D22B8
:1014A800120A3B120D44120E98120AD8120B3D1262
:1014B8000B4E120C0A306935206B3285615E8561EE
:1014C8005F855D6475650179327A0AC3E5349940B0
:1014D8000FC269D26A8A33755EFF755FFF0214F521
:1014E800C3E55994014003021403021530306A1B06
:1014F800206B18E533147004C26A61F7F533C3E54D
:101508005994014003021403021530C3E55C948228
:101518005016307404E529600FC3E53B78F0306B52
:101528000278609850028103C2AF120F047887E6F0
:10153800FE7602120F767887EEF6E4F522F523F5AB
:1015480024F525F562C268D2AF1206CF120F043017
:101558007406E529700201E441F1901A0D78201211
:1015680015E6E520B45A0CA31215E6E520B4A50348
:10157800021584120F161215A40215A3901A0378E7
:10158800807B0A1215E6A308DBF9901A0F788C7B8A
:10159800151215E6A308DBF9901A2422C2AF121619
:1015A800251215FF901A00740D1215EBA374021280
:1015B80015EBA374131215EB901A0378807B0A12AB
:1015C80015EAA308DBF9901A0F788C7B151215EA37
:1015D800A308DBF9121638121616901A2422E4937F
:1015E800F622E6438F01538FFD75EF0275B7A57597
:1015F800B7F1F0538FFE22438F02438F0175EF023C
:1016080075B7A575B7F1901A0DF0538FFC22901A93
:101618000D745AB1EB901A0E74A5B1EB227A307999
:10162800D07820901A40B1E6E520F709A3DAF7222E
:101638007A3079D0901A40E7B1EB09A3DAF922ABF6
:1016480071A872BB01027984BB02027985BB0302CF
:101658007986BB04027992BB05027987BB060279B9
:101668009CBB07027988BB08027989E8F7227C05C8
:101678001206E8DCFB22C2AF1206F81206FF1207B8
:101688000612070D1206D91206F81206FF120706EF
:1016980012070D1206D91206F81206FF12070612D3
:1016A800070DD2AF22C2AF12070D1207061206FFAE
:1016B8001206F81206D912070D1207061206FF12B3
:1016C80006F81206D912070D1207061206FF1206AF
:1016D800F8D2AF22AE71AF72C2AF1206F81206F896
:1016E8001206F81206D9DEF212070D1206D9DFF833
:1016F800D2AF22D17ED176D176757101757201751E
:101708007300D1DC7C05AD591206E8C3ED9559701C
:10171800F5C3E5599401400AC3E55994FF403202E4
:101728001737D147B1A4D17EC2AF75EF12D176DC9D
:10173800D50573C3E5739403500280C6D17605724C
:10174800E5711490009A93F808C3E57298500280E6
:10175800AED176D1760571C3E57194095002809CAB
:0C176800120F16B1A4C2AF75EF12D176BB
:101A00000D0213FFFFFFFF0304080101015AA501A6
:101A1000FFFFFFFFFF03FFFFFF25D0FAFA04FF01DE
:051A2000007AFF01FF48
:101A4000235467794B4637304148562320202020C5
:101A500023424C48454C4923463331302320202033
:101A60002020202020202020202020202020202076
:101C0000C2AFC2D353D9BF7581C043B20343FF8073
:101C1000752438752503B1BF75EF0275E24043F1B5
:101C20000853A4F7D283780379E67C1075220075F7
:101C30002300901DCC7B0675249875250130830206
:101C4000813D208308D8FBD9F9DCF781AD308308CA
:101C5000D8FBD9F9DCF781ADB17FE493A3C39A60D7
:101C6000028126DBDDB171600281267B08E493FAF4
:101C7000A3B152DBF87A30B152752200752300B15E
:101C800071EAFCEBFDC3ED94FE400EB1718A278B27
:101C900028ED30E0048A828B83B1717AC270D8C398
:101CA000ED94FE601050CEBD0022EC600675200061
:101CB0000200008100A827A9280809D804D90281B8
:101CC000C9B175EA89AAF281BB0D8199C3ED94036C
:101CD0005049EDA2E092007AC5C3E5829400E58305
:101CE000941C5093200010438F02438F0175B7A5B9
:101CF00075B7F1F030001FA827A9280809438F0104
:101D0000538FFDD804D902A11689AAE275B7A5752B
:101D1000B7F1F0A3A103538FFC81757AC1BD030C09
:101D2000E493A3FAB136DCF8B12E81758177AA224B
:101D3000AB23B152EBFAEA6222752608C3E52313FE
:101D4000F523E52213F52250066323A0632201D573
:101D500026EAB1BFB1BF75260AEAF4200102D28398
:101D6000300102C283B1BFC3134002C201D526EBCA
:101D700022B175EAFB208302A175308302A17A7536
:101D80002608AE24AF25C3EF13FFEE13FEB1C3B197
:101D9000BFC3EA133083024480FA30E703632201B1
:101DA000C3E52313F523E52213F52250066323A090
:101DB000632201D526D9E52265236523F52222AECB
:101DC00024AF250E0FDEFEDFFCD20122424C486517
:0A1DD0006C6934373132F31006015C
:00000001FF
